:020000040000FA
:060000000219FD02031CC1
:03000B0002008D63
:03001300020535AE
:03001B0002009050
:03002B000202D1FD
:03005B0002054457
:030073000203097C
:100080000406080C10182030406080A0C0054032E3
:10009000C2AFC2A853E6EFC28E856B8BC0D0D2D35D
:1000A000C0E0C0F0C2CAA8CCA9CDD2CAD2AF758A6E
:1000B00000C3E8956CF8E9956DF9C3E913F9E81305
:1000C000F8E5666007C3E913F9E813F8E97025E875
:1000D000956E4020956E501CE582B410177C007B15
:1000E000007A007908900000A86AE5667004C3E809
:1000F00013F801FD900000D2A8D2AA61E7E0FDC389
:100100009CC39840EF98EB33FB0582E0FCC39DC392
:100110009840E198EB33FB0582E0FDC39CC3984017
:10012000D398EB33FB0582E0FCC39DC39840C59890
:10013000EB33FB0582E0FDC39CC39840B798EB33DB
:10014000FB0582E0FCC39DC39840A998EB33FB05F7
:1001500082E0FDC39CC398409B98EB33FB0582E093
:10016000FCC39DC398408D98EB33FB0582217890AA
:100170000000D2A8D2AA61E7E0FDC39CC39840EF7B
:1001800098EA33FA0582E0FCC39DC39840E198EAFF
:1001900033FA0582E0FDC39CC39840D398EA33FA52
:1001A0000582E0FCC39DC39840C598EA33FA0582F6
:1001B000E0FDC39CC39840B798EA33FA0582E0FC9F
:1001C000C39DC39840A998EA33FA0582E0FDC39C19
:1001D000C398409B98EA33FA0582E0FCC39DC3981C
:1001E000408D98EA33FA0582EBC46B6A54F0F9EA61
:1001F000C454F0C3996009900000D2A8D2AA61E764
:10020000EBF4C454F0F9EAF4C4540F49FAEBF4C423
:10021000540FFBC3EAF99460FAEB9400FB5020C33F
:10022000E97B007A0079006016C3135006F9C39584
:1002300052600AE9F5527553007900800205533087
:100240003A27C3EA94D0F8EB9407F9400BE8FAE9AF
:10025000FB203509D235415D303502C235203902E7
:10026000B235C3EA33FAEB33FBEB2B3B3BF9C3EB81
:1002700013FBEA13FAEA29FAEB3400FB30E3047AC1
:10028000FF7BFFE5255403601B202A18E55D33F949
:10029000EB7007C3E99A4002E9FAE53CC4332AFA55
:1002A000EB3400FBC3EA33C4540FF8EB33C454F00F
:1002B00048F87005EA60027801900000D2A8D2AA3E
:1002C000E5226002152281D4900000D2A8D2AA6152
:1002D000E7C0D0C0E0C2CF0541E5666009E56560D2
:1002E000057565006104756501E52360021523C38A
:1002F000E55460057555006104E5552401F5555038
:10030000037555FFD0E0D0D032C2AF53E67F75926F
:10031000FA7593FFC22053917FD2AF32C0E0E58AD5
:10032000303408856B8BF0A3D0E032D0E0C2AF53FD
:10033000E6EFC0D0C0E0C0F0D2D3D2AF5388EFA870
:100340008AA98CAA40308D010A758A00758C0075C7
:100350004000438810E566700AC3E833F8E933F9D2
:10036000EA33FA30331FE8C4540FFAE9C454F04AB0
:10037000FAC3132AFAC3E833F8E933F9E82AFAE9A9
:100380003406FB61D830320FC3E833E933FAE82A88
:10039000FAE93400FB61D8303115E875F056A4AAAB
:1003A000F0E975F056A42AFAC5F03400FB61D8C311
:1003B000EA13FAE913F9E813F8E875F056A4AAF07D
:1003C000E975F056A42AFAC5F03400C313FBEA130A
:1003D000FAC3EB13FBEA13FAC3EB94125009C3EA16
:1003E0009434EB940750160522E52270021522C3BF
:1003F000E52294325002A128755400A12BE5226019
:100400000215223036067C007D088117AC31AD32F2
:10041000303A04AC33AD34C3EA9CFAEB9DFB92084E
:10042000AE60AF61303A425007203509D235813590
:10043000303502C235303504AE62AF63203902B2C6
:1004400035C3EA33FAEB33FBA208500AEAF424017D
:10045000FAEBF43400FBC3EA9450FAEB9400FB503F
:100460001478007A007B008175A208500878007A21
:10047000007B0081D4E5255403601B202A18E55D2C
:1004800033F9EB7007C3E99A4002E9FAE53CC4335B
:100490002AFAEB3400FBEA8EF0A4F9AAF0EB8EF016
:1004A000A42AFAC5F03400FBC3EB13FDEA13F8C32A
:1004B000ED13FDE813F80FEF146004C3E833F8C33D
:1004C000E933EA33FAEB33FBDFEDEB30E30678FF99
:1004D0007AFF7B078854D230E86003755500C3E586
:1004E0005BFC955C4002AC5CC3EC95545008EC7529
:1004F000F008A4FAABF0EAF4F8EBF45407F9C3E817
:10050000943CFAE99400FB50047A007B00885689F9
:10051000578A588B5975230AD0F0D0E0D0D053F7C2
:10052000DF43F74043E6103275230AD0F0D0E0D025
:10053000D043E61032C2AAD28EC2CA85CC6C85CD19
:100540006DD2CA32C2AFC0D0C0E0D2D3A8F9E55A4A
:1005500030E20AE5FA20E23520E132A165E5FA3021
:10056000E22B20E128C3E55713F8E55613F5FB8885
:10057000FCC3E55913F8E55813F5E988EA85575A9D
:1005800053F7BFD2A8303402D2AA53E6EF53F7DFB5
:10059000D0E0D0D0D2AF32790180147903801079C5
:1005A0000A800C791E80087964800479C8800078FC
:1005B00017E4D5E0FDD8FAD9F62278FF202828796B
:1005C000A1E76023E548601F74FF8548F084853FFC
:1005D000F030290375F005A4F8C5F0600278FFC378
:1005E000E8955D5002A85D885C22C3E54794A0E5CC
:1005F000489400E55C500314A1FB046002F55C2202
:1006000075E89022055EC3E55E9408405330EDF432
:10061000A8BDA9BE755E00E9FA79A0E76041EA705D
:1006200006E55F6018800CC3E8955F600EE55F50DB
:1006300005600A1480070460FA8002E55FF55FC375
:100640009569401B755BC0C394044013755B80C300
:100650009404400B755B40C394044003755B002217
:10066000E55B2410500274FFF55B22743279A68793
:10067000F0A4C5F0A2F733F55D227547007548F088
:1006800022C2AFC2CAA8CCA9CDAA4130CF010AD29A
:10069000CAD2AFC3EA13FAE913F9E813F8AB42ACD4
:1006A0004388428943C3E89BF8E99C20280A547F89
:1006B000F9302C02E19FC1F8AD448A44F9EA9D5417
:1006C0007FFA600678FF79FFC1DDAE45AF468B4506
:1006D0008C46A842A943C3E89EF8E99FF9C3E548C0
:1006E00013FBE54713FAE82AF547E93BF5485006BE
:1006F0007547FF7548FFE145AA47AB48AC47AD4891
:100700007E047F02C3EB9404400D1E1FC3EB9408CC
:1007100040052029021E1FC3ED13FDEC13FCDEF77C
:10072000C3EA9CFAEB9DFBEF6009C3E913F9E813F8
:10073000F8DFF7EA28FAEB39FB8A478B4850067B4B
:10074000FF8B478B48C3EB94025002D22C30280415
:100750007F03E1707892E6FFC3E53D948240110F7C
:10076000C3E53D94A040010FC3EF940640027F050E
:100770007E02E548C4540FF9E548C454F0F8E54753
:10078000C4540F28F8C3E89EFAE99400FB4009C35B
:10079000EA9401EB940050047A01E4FB0207EBAA0F
:1007A00047AB48EBC4FEEAC4540F4EFCC3EA9CFAC4
:1007B000EB9400FBC3E813C313F8EA28FAEB340008
:1007C000FB8A478B48C3EB94024002C22C7802EBB1
:1007D000C4FE7B00EAC4540F4EFAC3EA98FA4005FF
:1007E000C3940150027A017892E6FF302002E1EBD7
:1007F000854E92854F93D22043E680C3E49AF8E475
:100800009BF9C3E833F8E933F9302C03020880E898
:10081000FAE9FBD3E913FDE813FC884E894FC3EFD7
:1008200094036038EF20E00CE82CF8E93DF9ECFA8D
:10083000EDFB8013E828F8E939F9C3E82401F8E969
:100840003400F97AFF7BFFC3EF9403400F8A508B8B
:1008500051884A894B8C4C8D4D0208B5885089517E
:100860008A4A8B4B8C4C8D4D3028127550F0755147
:10087000FF754CF0754DFF754EF0754FFF0208B5D2
:10088000E8FAD3E813FC884EC3EF94036021EF200D
:10089000E007E82CF8ECFA01A0E8282401F87AFF38
:1008A000C3EF940340098A50884A8C4C0208B588EB
:1008B000508A4A8C4C30200201B5753A02D220434E
:1008C000E680E5255403602DA847A948C3E913F93C
:1008D000E813F8302804E92440F9C2AF53E67F75E5
:1008E0009100C3E498F594E499F595759104D220AC
:1008F00043E680D2AF22D221754900752000302B0B
:10090000037520402114D221754900752040302BF9
:100910000375200078017901202C20E5255403601F
:1009200002C2217914E548C313700104F8C394147A
:1009300040027814302804781B791BC3E833F8C3CD
:10094000E933F9202010E549600C302803D53A043A
:10095000D22221C711BD0549E59B5440B520022193
:10096000B130280908C3E899400118214320210A21
:1009700008C3E899400221142143C22153E67F7540
:100980009100302C117594007595F0759104D2206A
:1009900043E680020914E5487EFFC3334009C333B0
:1009A0004005C3334001FEC3E49E759400F59521D4
:1009B0008BC3E5399401500221143021022114D84F
:1009C0000221C52143C222C2AF53E67F7591008543
:1009D0005094855195759104854A92854B93D22008
:1009E00043E680D2AFE5255403600720290205398C
:1009F000801030220D202B0A20210715811581023D
:100A000013CA2278003021027801E53D75F007A471
:100A1000F9E5F028F5F0E9A2F013A2F113A2F21320
:100A2000F53DC394785003753D78C3E53D953E4050
:100A300009C290C291C29275D57F302002413A8599
:100A40004C92854D93D22043E68022203810C2AFCD
:100A5000C294D29375D51BD2AF759F23611BC2AFD1
:100A6000C294D29575D536D2AF759F23611B2038BD
:100A700010C2AFC29275D52DD293D2AF759F1361BC
:100A80001BC2AFC29075D52DD295D2AF759F0361B1
:100A90001B203810C2AFC293D29575D52DD2AF7539
:100AA0009F038077C2AFC295D29375D52DD2AF7513
:100AB0009F138067203810C2AFC29175D536D2958A
:100AC000D2AF759F238054C2AFC29175D51BD2930C
:100AD000D2AF759F238044203810C2AFC295D29404
:100AE00075D536D2AF759F138031C2AFC293D29401
:100AF00075D51BD2AF759F038021203810C2AFC2BD
:100B00009075D51BD294D2AF759F03800EC2AFC231
:100B10009275D536D294D2AF759F13227A147B7812
:100B200080127A107B8C800C7A0D7BB480067A0B55
:100B30007BC88000E564D5E001227902E4C294D547
:100B4000E0FDD291D5E0FDC291D5E0FDD294D5E093
:100B5000FDE920E002D29030E002D292E564D5E0D7
:100B6000FDE920E002C29030E002C2927496D5E026
:100B7000FDD9C9EAF8D5E0FDD8FBDBB8C29422C2A2
:100B800090C291C292C293C294C29575D57F2278C9
:100B90008076FF0876FF0876FF0876FF0876FF0864
:100BA00076FF0876090876FF087601788C760108CA
:100BB00076FF0876FF0876FF0876FF0876FF08764E
:100BC000030876FF0876FF0876FF0876250876D0BA
:100BD0000876280876500876040876FF087602081A
:100BE00076FF08767A0876FF087607087601087699
:100BF000FF0876FF08760008760022FA75F00CA44C
:100C0000ABF0EAC333F8740133F9E8C333F8E933DE
:100C1000F9E8C32BF8E93400F9E8C333F8E933F90C
:100C2000227888E6C39403D23A5002C23AC238E628
:100C300030E102D238A23892397886E614900080EA
:100C40009378A6F67886E6F53FC394025003753F85
:100C500002789CE6753EFFB40203753EA0B4030320
:100C6000753E8278A0E6F8600674282409D8FCF561
:100C7000697896E671FB88318932789EE671FB8847
:100C80003389347897E671FB88358936717F223055
:100C900036117A007B007CFF7D007E0091F58B6130
:100CA0008A6022303A227896E6FA7B00789EE6FC4B
:100CB0007D00C3EA33FAEB33FBC3EC33FCED33FDC9
:100CC0007E0A91F58B638A627896303A02789EE6C6
:100CD000FA7B007897E6FC7D007E00303A10C3EA8C
:100CE00033FAEB33FBC3EC33FCED33FD7E0A91F5B5
:100CF0008B618A6022C3EC9EFCED9400FDC3EC9AEC
:100D0000FCED9BFDC3EC9423ED940050047C237D0B
:100D100000C3EC94FFED940140047CFF7D017BFF58
:100D20000B7A000AEA7009C3EC33FCED33FDA12015
:100D3000EC8AF0A4AEF0ED8AF0A42E947C40E4EAB4
:100D4000F460DD22D236918F1205A31205A37A003A
:100D50007B007C1012059BE5542AFA74003BFBDCF7
:100D6000F37C04C3EB13FBEA13FADCF7FFEB60023E
:100D70007FFFC236918F2278A5E6F95403C28570B1
:100D800002D285E9540CC2867002D286E95430C280
:100D9000877002D287E954C07000227567007568B9
:100DA000007597DE7597AD7581C043FF8075EF06BE
:100DB00075A900717F7580FF75F1F075A4E07580ED
:100DC000FF75D4FF75900075F23F75A53F759000D3
:100DD00075D53F75A60175E34075E202717FE4F8B1
:100DE000F6D8FD718F12140E78988664753001C2A2
:100DF000AF1205AB711C1205A371221205A3712855
:100E00001205A3B177C2AF75670075680078FA79EB
:100E1000FA308407D9FBD8F7021C009121918F7812
:100E2000988664717F75A91375A71075C10075A7A1
:100E30000075660075E404758811758E047589095E
:100E400075C80475910475D84075D90875F7827511
:100E50009E0375960275DA4275DB4275A82375E626
:100E60009075B801759B80759D0075D10C75BCB9E6
:100E700075BB1075E88075B201120597D2AF753C4D
:100E800000C2301205ABC231C232C233C234755215
:100E9000007522001205A7C3E522940A5002E168FA
:100EA000D2317522001205A7C3E522940A5002E14F
:100EB00068C231D2327522001205A7C3E522940A16
:100EC0005002E16875E4C4758851758E017589AA70
:100ED000758C00758D00C2A9D2ABD2AA756B8075D6
:100EE0006A14756E50C232D23475220A1205A77583
:100EF0006A10C3E522940A75520075530040697563
:100F00008E0C756B00756A28756E2875220A12059D
:100F1000A7756A20C3E522940A75520075530040F4
:100F200047758E0C756B80756A14756E1475220A80
:100F30001205A7756A10C3E522940A75520075530D
:100F400000402575E404758811758E04758909D2F1
:100F5000A9C2ABC2AAC234D2337522001205A7C3FC
:100F6000E522940A4002C10512059B203003020EBF
:100F700005C2AF711C711C711CD2AF1205AB2034BD
:100F800003303A0302102712059B788CE6C39401C4
:100F90005003021027E530C3940150030210277557
:100FA00067A57568F17F02D236918F1205A7C2AF8F
:100FB000C236918FC3E554947FD2AF406A12059731
:100FC000C2AF712ED2AFDFDFB144C3EF7897F61214
:100FD00005AB1214FB7F0AD236918F1205A7C2AF60
:100FE000C236918FC3E554947FD2AF50E812059773
:100FF000C2AF711C12059F711CD2AFDFDAB144EF92
:1010000024037896F6F87997E7C394234003985021
:1010100006E824237897F61205AB9155B12A1205FC
:10102000A7120C8F020E057567007568001205A7E0
:10103000C3E55494014003020F7EC2AF120B2E127F
:101040000B2E120B2ED2AF1205AB753000E4F53724
:10105000F5380537E537F4703F0538789AE67819A2
:10106000146012783214600D787D14600878FA14D8
:101070006003753800C3E53898401D120B7F1205D8
:1010800097153875370078998664C2AF120B2ED247
:10109000AF789886641205A712059FE523700302B6
:1010A0000E05C3E55294015014C3E554940140A2C7
:1010B0001205A7E5237003020E0502125BC3E55279
:1010C00094017017C2AF120B7F78998664120B1CC3
:1010D00078988664D2AF1205A7414DC3E5529402B9
:1010E0007017C2AF120B7F78998664120B22789822
:1010F0008664D2AF1205A7414DC3E5529403701721
:10110000C2AF120B7F78998664120B287898866498
:10111000D2AF1205A7414DC3E55294047013C2AF7C
:10112000120B7F78998664120B2ED2AF1205A7415D
:101130004DC3E55294057017C2AF120B7F789986A4
:1011400064120B2E78988664D2AF1205A7414DC366
:10115000E55294077019C3E5539409500201A27433
:1011600001303A0274037888F6C238C239414DC35F
:10117000E55294087019C3E5539409500201A27412
:1011800002303A0274047888F6D238D239414DC31D
:10119000E55294097017C3E5539409500201A23037
:1011A0003A0BC37888E69402F6C23A414DC3E55241
:1011B000940A7016C3E5539409500201A2203A0A1A
:1011C0007888E62402F6D23A414DC3E55294147071
:1011D00025C3E5539409500201A2C2AF901A0B74C3
:1011E0000093D2AF7888F613C238C2394002D238A1
:1011F0004002D2398057C3E55294157038C3E55385
:101200009409404FC2AF901A0B740093D2AFF8B854
:1012100001027402B802027401B803027404B80433
:101220000274037888F613C238C2394002D23840BB
:1012300002D2398018C3E552940C70117567A575F8
:1012400068F1C3E5539409400A9155D2AF75520035
:1012500075530075670075680001A2C2AF120B7F5D
:10126000E4D2AFE4F55EF524F525F53D755E081290
:10127000059712060030EDFDA8BDA9BEE97001F882
:10128000885F120604755E08C2AF12066B855D5B4F
:10129000855D5CD2AF75A71075C13075A70075A9C3
:1012A00003756601303A07C238303502D238D22889
:1012B000753900120AD7120AFA12067A120681123A
:1012C000067A12068112067A120906120A03120A17
:1012D0004B1206811208F6202C031205BA302C039B
:1012E0001205EA120A03120A6E1206811209061288
:1012F0000A03120A911206811208F6120A03120A50
:10130000B4120681120906120A03120AD7120681C4
:101310001206001208F6120A03120AFA1206041242
:101320000681302827855D5B79187A0CC3E53999E9
:10133000400EC228D2298A3B855D5B855D5C800CAE
:10134000C3E554940140030212C861D230291F2022
:101350002B1CE53B147006C229D22A41C8F53B205C
:101360003A07C3E554940140030212C88064753CF7
:1013700000203A0F78FA79A4E760027803C3E555B4
:1013800098504FE523604B303A1720380520350739
:10139000800F303502800A202B07D22B855D5B4100
:1013A000F878F0302B05855D5B7820C3E5489850D0
:1013B000030212C8302B1BC22BC238303502D23880
:1013C000D229753B12855D5B41C8053CE55460023E
:1013D00061D5753C00C2AF120B7F752400752500E6
:1013E00075A91375A71075C10075A700756600D2A1
:1013F000AF1205A7120B7F78A4E66006D293D294B1
:10140000D295C3E53C94044003020E05014D901AA9
:101410000D7820918EE520B4550AA3918EE520B475
:10142000AA0280137567A57568F1120B8F91557527
:101430006700756800801D901A0378807B0A918E82
:10144000A308DBFA901A0F788C7B1A918EA308DB25
:10145000FA901A2922C2AF91D191AE901A0074105D
:101460009193A3743E9193A374219193901A03785E
:10147000807B0A9192A308DBFA901A0F788C7B1A72
:101480009192A308DBFA91E491C2901A2922E49385
:10149000F622E6438F01538FFDFFC3E583941C4082
:1014A0000122EF8567B78568B7F0538FFE22438F1F
:1014B00002438F018567B78568B7901A0DF0538F87
:1014C000FC22901A0D74559193901A0E74AA919360
:1014D000227A3079D07820901A40918EE520F70951
:1014E000A3DAF7227A3079D0901A40E7919309A3D2
:1014F000DAF9227C051205ABDCFB22C2AF120B1C11
:10150000120B22120B28120B2E12059F120B1C120B
:101510000B22120B28120B2E12059F120B1C120B02
:1015200022120B28120B2ED2AF22C2AF120B2E1298
:101530000B28120B22120B1C12059F120B2E120BE2
:1015400028120B22120B1C12059F120B2E120B28B5
:09155000120B22120B1CD2AF2277
:1019FD00020D9B103E21FFFFFFFFFFFF09FF01FFBF
:101A0D0055AA01FFFFFFFFFF03FFFFFF25D0285061
:0D1A1D0004FF02FF7AFF0701FFFF0000FF3A
:101A4000234A5F485F33302320202020202020209D
:101A500023424C48454C492445464D3842323123B7
:101A60002020202020202020202020202020202076
:101C0000C2AFC2D37597DE7597AD7581C075A90057
:101C100043FF80752438752503B1DB7529A5752A26
:101C2000F143F11053A4EFD28475D4FF75E3407DE6
:101C3000FA780379E67C10752200752300901DE880
:101C40007B0675249875250130840281482084081C
:101C5000D8FBD9F9DCF781BA308408D8FBD9F9DC94
:101C6000F781BAB19BE493A3C39A6004DDC381BA40
:101C7000DBDBB18D600281317B08E493FAA3B16EA6
:101C8000DBF87A30B16E752200752300B18DEAFC65
:101C9000EBFDC3ED94FE400EB18D8A278B28ED300D
:101CA000E0048A828B83B18D7AC270D8C3ED94FE32
:101CB000601950CEBD0029EC600F7520007521FF22
:101CC000752900752A000200008100A827A92808AC
:101CD00009D804D90281DDB191EAF281D10D81A642
:101CE000C3ED94035051EDA2E092007AC5C3E582A2
:101CF0009400E583941C508C200010438F02438F86
:101D0000018529B7852AB7F0300027A827A9280818
:101D100009438F01538FFDD804D902A132C3E58353
:101D2000941C4003A3A117E28529B7852AB7F0A325
:101D3000A117538FFC81827AC1BD030CE493A3FAEF
:101D4000B152DCF8B14A81828184AA22AB23B16E00
:101D5000EBFAEA6222752608C3E52313F523E52290
:101D600013F52250066323A0632201D526EAB1DBD6
:101D7000B1DB75260AEAF4200102D284300102C2E6
:101D800084B1DBC3134002C201D526EB22B191EA34
:101D9000FB208402A191308402A196752608AE240E
:101DA000AF25C3EF13FFEE13FEB1DFB1DBC3EA13C0
:101DB0003084024480FA30E703632201C3E5231331
:101DC000F523E52213F52250066323A0632201D5F3
:101DD00026D9E52265236523F52222AE24AF250E00
:101DE0000FDEFEDFFCD20122424C48656C693437BD
:061DF0003164E8B20601B7
:00000001FF
